:1000000000308A004C2B0000CA00030ECB009A304F
:1000100081079E185228A008031D1328061B1228CA
:10002000A00A9F01522820080A3C031D40289F0A6D
:100030001F08043C031D3628061F3528A00121088F
:100040000A3C031D25289E1435281C08133C031C5C
:1000500034282108203C031833281C089C0A1B075D
:1000600084002108800035281E143F281F08053C05
:10007000031D3F28061F3E28A0013F289F0352284A
:100080009F0A1F08083C031D4828A00A9F01522808
:100090001F08043C031D5228061B5028031051283A
:1000A0000314A10CA308031D5F289D0803195E28F3
:1000B000A30AA20186131D08A4009D017D28A20A9F
:1000C0002208073C03187D28A201A30A23080A3C42
:1000D000031D702886179D08031D6F281E157D2897
:1000E00023080B3C031D7628A3017D280310A40CD4
:1000F00003187C2886137D288617A0308B054B0EAD
:100100008300CA0E4A0E090009000A108A100A115B
:100110008207AD34033438340534B9340234B93489
:100120000434B934023438340534B9340234C534B3
:10013000053402340334B93404340234033438341B
:10014000053402340334C534053454340334B9342B
:100150000434543403343834053454340334C5344B
:100160000534B93402346134063402340334613462
:1001700006345434033461340634AD34033461340A
:100180000634AD340334B9340434AD340334C534E7
:1001900005342530840000080319DD2801308D0066
:1001A0008C018C0BD1288D0BD0284A308C008C0B05
:1001B000D72800000000800BCE28672B9D08031D68
:1001C000DE281E1140089D0000341030C9008C014B
:1001D0008F01C60CC50C031CF32847088C070318B5
:1001E0008F0A48088F078F0C8C0C8E0C8D0CC90B56
:1001F000E928003425309B008B161E100D30C000FE
:10020000DE200A30C000DE201E1C17291E104530DB
:10021000C000DE205230C000DE205230C000DE20A0
:100220004F30C000DE205230C000DE201D294F308C
:10023000C000DE204B30C000DE200D30C000DE20CC
:100240000A30C000DE209E109C01B9019E18992939
:100250001C083902031835293908B90A253E8400DB
:100260000008BF00C000DE2028299C08031D392992
:1002700026292508BA001C0839020318482939081C
:10028000B90A253E84000008BF00C000DE203B29DB
:100290003A082F3C031853293A08393C031C5329C8
:1002A0003030BA0278293A08403C03185E293A08EF
:1002B000443C031C5E293730BA0278293A08603C76
:1002C000031869293A08643C031C69295730BA02AB
:1002D00078293A082A3C031D70290E30BA00782983
:1002E0003A08233C031D77290F30BA0078292629C4
:1002F0003A0D8C008C0DFC308C050C08BF000C0AEC
:1003000085208F003F08852093000F0894003A0D48
:100310008C008C0DFC308C050C08023EBF003F0A9F
:1003200085208F003F08852095000F0896009929A9
:1003300026291E1C9C29FE289E189F29AB2A2530A1
:10034000BB001E141C08023C031CA729FE2825081C
:10035000533C0319B0292508733C0319B029FE2822
:100360002608303C0318B8292608323C0318B9295E
:10037000FE2827083D3C031D162A2830BB00BD017E
:10038000BC011C089C03033C0318DB293D08C60084
:100390003C08C500C8010A30C700E5200E08BD00B2
:1003A0000D08BC003B08840030300002BC07031875
:1003B000BD0ABB0AC1292608313A0319E329033AC9
:1003C0000319FA29152ABD08031DEA293C08273C10
:1003D0000318F9293D080B3C031CF929031DF429D6
:1003E0003C08B83C031CF9293D0898003C089700DC
:1003F0001E10152A3D08023C0318142AFF3A031D5B
:10040000052A3C08833C0318142A3D08043C031CBD
:10041000142A031D0F2A3C084C3C031C142A3D08D7
:100420009A003C0899001E10152AAA2A27083F3C6A
:10043000031DAA2A1C08033C03191F2AAB2A2608FD
:10044000313A0319272A033A03192C2A312A1808AA
:10045000BD001708BC00312A1A08BD001908BC00ED
:10046000312A0D30C000DE200A30C000DE205330BB
:10047000C000DE202608C000DE203D30C000DE20A7
:100480003D08BF003C08BE002530C0000130C1005F
:10049000C3010A30C20043083F02031C632A031D44
:1004A000552A42083E02031C632AC10A4308C600BB
:1004B0004208C500C8010A30C700E5200E08C30085
:1004C0000D08C2004B2AC1080319972A0130C40045
:1004D000C301C2004108440203187C2AC40A43082D
:1004E000C6004208C500C8010A30C700E5200E0852
:1004F000C3000D08C2006A2A400884003030800022
:1005000043083F02031C942A031D8A2A42083E0224
:10051000031C942A4208BE024308031C430FBF0277
:1005200040088400800A802AC00AC103632A400868
:10053000840080012530BB003B088400800803193B
:10054000A92A3B0884000008BE00C000DE20BB0AC8
:100550009C2A1E10FE281E1DAB2A8B126F2B2030EA
:10056000C000BC01BD01BE01BF0137088F003608C5
:100570008E0035088D0034088C0003100C1CCE2A28
:100580003808BC0739080318390FBD073A080318A3
:100590003A0FBE073B0803183B0FBF07BF0CBE0C4A
:1005A000BD0CBC0C8F0C8E0C8D0C8C0CC00BBD2AA2
:1005B000302B8C018D018E018F01BD01BE01BF0169
:1005C000C0013C083B043A0439040319172B2030BE
:1005D000C1000310B50DB60DB70DB80DBD0DBE0DA4
:1005E000BF0DC00D3C084002031D002B3B083F021D
:1005F000031D002B3A083E02031D002B39083D0263
:10060000031C112B3908BD023A08031C3A0FBE0225
:100610003B08031C3B0FBF023C08031C3C0FC002FD
:1006200003148C0D8D0D8E0D8F0DC10BE92A00006A
:100630003D308400472BB301B2012F08B1002E08D2
:10064000B0003308B7003208B6002F08B5002E08F6
:10065000B400BB01BA011A08B9001908B800AF2AE2
:100660000F08B4000E08B3000D08B2000C08B1006A
:100670000F08B8000E08B7000D08B6000C08B5004A
:10068000BC01BB010430BA005630B900D92A0D08AC
:100690008E000C088D00003484011F3083055F300C
:1006A00097009801E830990003309A009C019D0161
:1006B0009F01A001A101A201A301A40100306500D6
:1006C00040306600803086006430A500C92883165B
:1006D0000108C7390838810083128B17FA288A234A
:0406E0006E2B63001A
:0C071400A50104301702AE001808AF0069
:100720000030031C0130AF022F08C6002E08C500A0
:10073000C8011230C700E5200E0892000D08910094
:10074000A701A6011408AF001308AE001B230E0872
:10075000A9000D08A800AB01AA011608AF001508F2
:10076000AE001B230E08AD000D08AC00910A920AE2
:1007700003308A0088308400250E0F39820700007C
:100780000000000000000000000000000000000069
:1007900000000000000000000000000086150F3C73
:1007A00082070000000000000000000000000000C0
:1007B0000000000000000000000000000000000039
:1007C00086110F30A50527083F3989000014080855
:1007D000A5072B083F39890000140808A507280839
:1007E000A6070318A70A2908A7072C08AA070318B1
:0E07F000AB0A2D08AB07910BFE2B920BBC2B16
:0207FE000034C5
:104200000000000001000300050007000A000E0086
:10421000120016001B00200025002B003000360085
:104220003C00420048004D00530058005D00620011
:1042300066006A006E0071007300750077007800F8
:104240007800780077007500730071006E006A00D6
:10425000660062005D00580053004D0048004200B7
:104260003C00360030002B00250020001B0016000B
:1042700012000E000A000700050003000100000004
:02400E00F13F80
:00000001FF
